:100000000C94CE020C9412030C9412030C94120361
:100010000C9412030C9412030C9412030C9412030C
:100020000C9412030C9412030C94040E0C94D60E30
:100030000C9412030C9412030C9412030C941203EC
:100040000C9412030C94E0220C9412030C941203EF
:100050000C9412030C94731C0C9412030C94120352
:100060000C9412030C9412030C9412030C941203BC
:100070000C9412030C9412030C9412030C941203AC
:100080000C9412030C9412030C9412030C9412039C
:100090000C9412030C9412030C9412030C9412038C
:1000A0000C9412030C9412030C941203430F650F6B
:1000B0005310650F5310AA0FCD0F53102210351097
:1000C000041304133313331369138913BA14BA14C2
:1000D0009413BA1444144414AB14BA14BA14B414D8
:1000E00051145114511451145114511451145114E8
:1000F00051145114511451145114511451145114D8
:100100006314701477147E1488140000F0A32E007A
:100110004C002A00E100015200001E0034000400DF
:1001200033000000E3001F00360012001400350009
:1001300028002000370008000D005000E2002100D8
:10014000130018000E004F00000022001C000C00DD
:100150001B0000004B000030290000002B000000B5
:100160004E00000039000000280000004A00230073
:1001700009000700050000004D0024000A000B00E4
:1001800010005200E6002500060017001A0051007A
:10019000E40026001500110019002F002C00270094
:1001A0000F0016001D0030000352310038002D00F2
:1001B000E500015200000100010001000100010002
:1001C00000003A001E0220022202010001003B0052
:1001D0001F0221022302010001003C002F0226021F
:1001E0002F00010001003D00300227023000010015
:1001F00001003E003102350035020000010001001F
:1002000001000000010000000100010001000000E9
:100210000100000001003F005200510024020000D4
:1002200001004000240021001E00010001004100E7
:10023000250022001F003700010042002600230095
:10024000200027000100430025022E0231002E006D
:100250000100440045000100010001000000000011
:100260000000000000000100000000001E0014005B
:1002700014000000000000001E001A00160000001C
:10028000190000001E000800070001000600000021
:100290001E00150009000100000000001E001C00E7
:1002A0001C000000000001001C0000001C000000F9
:1002B000000000001C0000001C0000000000000006
:1002C0001E001C001C000000000000001E001800A2
:1002D0000D000100000000001E000C000E000100D7
:1002E000100000001E0012000F00000011000000AE
:1002F0001E00130033000000010000001E002F004C
:1003000034000100000001000100010001000100B3
:1003100000000100010001000100010001000100D6
:100320000100F2000100010001000100F000F100F5
:100330000100F400010001000100F3000100F500DC
:1003400001000100010001000100000001000100A6
:100350000100000001000000010001000100000098
:100360000100000001000100010001000100000087
:1003700001000100B600AC000100A900010001006D
:100380000100AE000100AA00B6000100B700AB00FA
:100390000100A800010001000100010001000100AE
:1003A000010001000100010001000100000016032E
:1003B0004500720067006F0044006F007800200065
:1003C00045005A00000016034500720067006F00E8
:1003D00044006F007800200045005A00000004032C
:1003E000090409026D00040100A0FA0904000001DB
:1003F00003010100092111010001223F00070581CD
:100400000308000A09040100010301020009211187
:10041000010001224D000705820308000A090402B9
:10042000000103000000092111010001223600072C
:1004300005830308000A0904030001030000000902
:100440002111010001223900070584031000011267
:1004500001100100000008EDFE0713010001020079
:100460000105010906A101050719E029E715002585
:100470000195087501810205081901290595057581
:10048000019102950175039101050719002977155E
:10049000002501957875018102C005010980A1013F
:1004A000850216010026B7001A01002AB700751050
:1004B00095018100C0050C0901A101850316010009
:1004C000269C021A01002A9C02751095018100C029
:1004D00005010902A1010901A10005091901290568
:1004E00015002501950575018102950175038101AE
:1004F0000501093009311581257F950275088106AE
:1005000009381581257F950175088106050C0A3883
:10051000021581257F950175088106C0C005010976
:1005200006A101050719E029E715002501950875C1
:1005300001810295017508810105081901290595B8
:1005400005750191029501750391010507190029AF
:10055000FF150025FF950675088100C0000000000A
:1005600000000000000000010204060A0F17202C02
:100570003A4A5D71879DB3C7DAE9F5FCFFFCF5E9FE
:10058000DAC7B39D87715D4A3A2C20170F0A06041B
:1005900002010000000000000000000011241FBE46
:1005A000CFEFDAE0DEBFCDBF04B603FE24C08091FA
:1005B000FB019091FC01A091FD01B091FE018730FB
:1005C000904BA740B04BB9F41092FB011092FC0184
:1005D0001092FD011092FE0114BE84B7877F84BF84
:1005E00088E10FB6F89480936000109260000FBE0F
:1005F000E0E0FFE3099511E0A0E0B1E0EEE4F9E40A
:1006000002C005900D92A433B107D9F711E0A4E31D
:10061000B1E001C01D92AB3FB107E1F70E94480B6A
:100620000C94A5240C9400001092B9008AE08093E9
:10063000B800089594EA9093BC009091BC0097FF95
:10064000FCCF9091B900987F983021F0903111F053
:1006500081E008958093BB0084E88093BC00809182
:10066000BC0087FFFCCF8091B900887F883111F0F2
:10067000803471F780E0089584E98093BC00809114
:10068000BC0084FDFCCF08958093BB0084E8809378
:10069000BC008091BC0087FFFCCF9091B900987F8F
:1006A00081E0983209F480E0089584E88093BC00EA
:1006B0008091BC0087FFFCCF8091BB0008958091A2
:1006C0000101811115C080E40E941A038093010189
:1006D00081110CC082E10E944403809301018111C9
:1006E00005C08FEF0E944403809301010E943C03E8
:1006F00084B1807F84B985B1807F85B98AB1837FD9
:100700008AB98BB1837F8BB93E98469808950E9431
:100710001A05809301010E945F0380B38C7080BB37
:1007200081B3836F81BBA5E3B1E0E3E4F1E08EE048
:100730008E0F11921D928E13FCCF0C940405BF9264
:10074000CF92DF92EF92FF920F931F93CF93DF939D
:1007500080910101882379F0809134018F5F80932B
:100760003401811108C00E941A0580930101811192
:1007700002C00E94AC0405E311E0C0E0D0E0DD243B
:10078000D39482E0C82EEE24E394F12CC730D10537
:1007900000F580910101811164C080E40E941A0378
:1007A00080930101811112C082E10E944403809371
:1007B000010181110BC0C7010C2E01C0880F0A94E2
:1007C000EAF780950E944403809301010E943C0354
:1007D00048C0CA30A1F028F4C83059F0C93061F0DF
:1007E00005C0CC3089F070F0CD3089F0209A28987F
:1007F00010C0219A29980DC0229A2A980AC0239ADB
:100800002B9807C0529A01C0539A5B9802C03E9A37
:10081000469890EA9A95F1F79FB1799902C082E0E3
:1008200001C080E091709D25982B7C9902C084E0E6
:1008300001C080E0892B7D9902C038E001C030E022
:10084000832B7E9902C020E101C020E0822B9FB162
:100850009095991F9927991F9295990F907E892BB2
:100860000FC080910101811149C080E40E941A03E8
:1008700080930101882379F1B12C0E943C038B2DD8
:10088000F8019081981719F08083C09200010E94AE
:100890005F0321960F5F1F4FCE30D10509F076CF51
:1008A00080910001882361F18150809300018823A9
:1008B00039F08FE99FE00197F1F700C0000020C0F8
:1008C000A3E4B1E0E5E3F1E0CF01825F91919D9374
:1008D0008E13FCCF15C083E10E9444038093010175
:1008E0008111CACF81E40E941A0380930101811112
:1008F000C3CF0E945503B82EB094BFCF80E0C0CFC5
:100900000E94AA0481E0DF91CF911F910F91FF9087
:10091000EF90DF90CF90BF900895E82FF0E0ED5B6F
:10092000FE4F8081089508950F931F93CF93DF9317
:10093000C3E4D1E010E00C2F025F899190E00E94A7
:10094000991B180F0C13F9CF812FDF91CF911F91B5
:100950000F9108950C94B40556985E9825982D989B
:1009600026982E9827982F988FEF90E090938900E3
:100970008093880090938B0080938A0090938D00E1
:1009800080938C00259A2D9A2FEF80E792E02150DA
:1009900080409040E1F700C00000269A2E9A2FEF89
:1009A00080E792E0215080409040E1F700C00000D5
:1009B000279A2F9A2FEF80E792E0215080409040B5
:1009C000E1F700C0000025982D982FEF80E792E016
:1009D000215080409040E1F700C0000026982E98FA
:1009E0002FEF80E792E0215080409040E1F700C077
:1009F000000027982F9856985E9825982D9826984D
:100A00002E9827982F98089589EA8093800089E08E
:100A10008093810024982C983F988AB18F748AB96A
:100A20006E98479A8BB1806B8BB9769A0E94AC0412
:100A30000C94B30580E280930101809151018111F2
:100A40000EC00E94140381E0809351012FEF83EDCB
:100A500090E3215080409040E1F700C0000080E426
:100A60000E941A038093010181112EC00E94440349
:100A700080930101811128C00E94440380930101E9
:100A8000811122C08FE30E944403809301018111F0
:100A90001BC00E943C0380E40E941A038093010162
:100AA000811112C08CE00E944403809301018111E6
:100AB0000BC00E94440380930101811105C08FE3A4
:100AC0000E944403809301010E943C038091010134
:100AD0000895CF93DF93EC016091BD017091BE0149
:100AE0008091BF019091C0010E94A51BCD2BE9F020
:100AF000823021F082E00E94621903C082E00E94ED
:100B0000831988E00E94A81185E10E94A81189E05C
:100B10000E94A81189E10E94A81182E10E94A811F7
:100B20008FE0DF91CF910C94A81188E00E947012A1
:100B300085E10E94701289E00E94701289E10E9492
:100B4000701282E10E9470128FE0DF91CF910C94BD
:100B50007012611105C0FC01828190E00E9469055C
:100B600080E090E0089508950F931F938091BD0158
:100B70009091BE01A091BF01B091C0018C019D0177
:100B80000470112722273327AC01BD014870552777
:100B90006627772756985E9825982D9826982E9840
:100BA00027982F9881FF02C0259A2D9A012B022B9E
:100BB000032B11F0269A2E9A452B462B472B11F02A
:100BC000279A2F9A1F910F91089581E0089581E04F
:100BD00008950C94E70508950F931F93CF93DF9327
:100BE0008C01FC01C081D181CE010E941E1ABE0180
:100BF0000E949506EC01B8010E94E905882309F4DA
:100C00008DC0F8018281882309F44AC080915D017A
:100C100081111FC0C431F0E5DF0709F051C00E9407
:100C2000EB0581E080935D010E943D1C90935C0187
:100C300080935B011092540110925601109255015D
:100C4000109258011092570110925A0110925901B6
:100C500065C080915B0190915C010E94491C883CB9
:100C6000910570F480915401E82FF0E0EE0FFF1F22
:100C7000EB5AFE4FD183C0838F5F809354014EC0E7
:100C8000C43880E5D80721F0C538D04501F13AC015
:100C9000F8018281882341F01092520182E01EC047
:100CA000C438E0E5DE0759F580915201811106C094
:100CB00086E20E94A81186E20E94701282E01CC0A7
:100CC000C438F0E5DF0741F3C538D045D9F4F80161
:100CD0008281882331F01092530180E20E94BF127A
:100CE0001DC080915301811106C087E20E94A811A6
:100CF00087E20E94701280E20E94C6120FC0C538BF
:100D0000D04529F381E08093520180935301C801BB
:100D1000DF91CF911F910F910C94E50580E0DF9159
:100D2000CF911F910F910895089596E0799FF0015A
:100D3000112494E5899FE00DF11D1124E60FF11DAA
:100D4000EE0FFF1FE25FFE4F859194910895880F8B
:100D5000991FFC01E657F040859194910895880F02
:100D6000991FFC01E65FFE4F8591949108950F93C2
:100D70001F93CF93DF93EC01811520E3920750F589
:100D8000C11580E2D80708F0C3C0CB3BD10590F471
:100D9000C83AD10508F06AC0C53AD10508F05BC071
:100DA000C430D10508F0D0C1219709F0CAC101E0D3
:100DB00010E00AC2CF3FD10511F008F0C5C1C03F15
:100DC000D10508F0A2C0CE01805E9109089708F411
:100DD000BBC1B7C1C13090E5D90709F4A2C020F565
:100DE000C0318FE4D80770F4C11590E4D90708F03A
:100DF00094C0C11521E3D20708F0A3C1DD278E01FD
:100E0000106CE2C1C115D04509F09BC10E942515A7
:100E10008FEF94E32CE0815090402040E1F700C038
:100E200000000E94981CD0C1C11597E5D90758F45D
:100E3000C03121E5D20708F01CC1C43180E5D807D4
:100E400008F475C07EC1CE0190578115904108F01D
:100E500078C1DF7073C1C53AD10509F477C1C63ACC
:100E6000D10509F076C102E810E4AEC1C83AD10557
:100E700009F472C1C93AD10509F471C1CA3AD10560
:100E800009F470C1CB3AD10509F46FC1CC3AD10550
:100E900009F46EC1CD3AD10509F46DC1C03BD1054D
:100EA00009F46CC1CE3AD10509F46BC1CF3AD10532
:100EB00009F46AC1C13BD10509F469C1C23BD1053E
:100EC00009F468C1C33BD10509F467C1C43BD1052E
:100ED00009F466C1C53BD10509F465C1C63BD1051E
:100EE00009F464C1C73BD10509F463C1C83BD1050E
:100EF00009F462C1C93BD10509F461C1CA3BD105FE
:100F000009F460C100E014E45FC18E0110655CC1AA
:100F1000CE019F700E94AF0658C1DF708E01106A2B
:100F200053C18091DA0181608093DA014DC10E9442
:100F30003D1E811102C00E94231E0E945A1E90E095
:100F40009093FB018093FA01C23080E5D80721F429
:100F50008091FA01816086C0C43090E5D90721F400
:100F60008091FA0182607EC0C63020E5D20721F46C
:100F70008091FA01846076C0C83080E5D80719F402
:100F80008091FA0127C0CA3090E5D90721F48091F9
:100F9000FA01806167C0CC3020E5D20721F480914E
:100FA000FA0180625FC0CE3080E5D80721F48091DD
:100FB000FA01806457C0C03190E5D90721F48091CF
:100FC000FA0180684FC0C23120E5D20729F4809130
:100FD000FA018460886046C0C33080E5D80721F4F8
:100FE0008091FA018E7F3EC0C53090E5D90721F48B
:100FF0008091FA018D7F36C0C73020E5D20721F4F9
:101000008091FA018B7F2EC0C93080E5D80719F492
:101010008091FA0126C0CB3090E5D90721F4809168
:10102000FA018F7E1FC0CD3020E5D20721F48091D8
:10103000FA018F7D17C0CF3080E5D80721F4809169
:10104000FA018F7B0FC0C13190E5D90721F480915F
:10105000FA018F7707C0C331D04531F48091FA018E
:101060008B7F877F8093FA018091FA010E945E1E38
:10107000ABC08D2F99278F70992781309105D9F4B6
:101080009E012370332702C0880F991F2A95E2F72B
:101090009C688E0144E0000F111F4A95E1F700277C
:1010A0001370802B912B53E0CC0FDD1F5A95E1F785
:1010B000C076DD272FC08230910531F4DC2FCC279C
:1010C0008E01016F106A80C08330910569F4CE01F2
:1010D0008370992701E010E002C0000F111F8A956C
:1010E000E2F7C8019C680FC084309105B9F4CE01C5
:1010F0008370992701E010E002C0000F111F8A954C
:10110000E2F7C8019A6823E0CC0FDD1F2A95E1F7CA
:10111000C07ED7708C010C2B1D2B56C085309105DD
:1011200031F4DC2FCC278E01046F106A4DC0069776
:1011300009F04AC0CF71DD27DC2FCC278E01106269
:1011400043C000E010E040C08E013EC001E810E462
:101150003BC003E810E438C002EE14E435C009EEE9
:1011600014E432C00AEE14E42FC005EB14E42CC0E2
:1011700006EB14E429C007EB14E426C00CEC14E4DD
:1011800023C00DEC14E420C003E815E41DC00AE8F8
:1011900015E41AC002E915E417C004E915E414C007
:1011A00001E216E411C003E216E40EC004E216E404
:1011B0000BC005E216E408C006E216E405C007E22B
:1011C00016E402C00AE216E4C801DF91CF911F9134
:1011D0000F91089596E0799FF001112494E5899F7D
:1011E000E00DF11D1124E60FF11DEE0FFF1FE25F70
:1011F000FE4F85919491803E9105E0F4803C9105ED
:1012000058F58133910509F46FC048F4893291058E
:1012100009F463C08A32910509F46DC072C0893344
:101220009105E9F082389105D1F08533910509F4F3
:101230004DC067C0833E910581F138F4803E910531
:10124000B9F0823E9105D9F05CC0863E910561F10E
:10125000873E9105A1F155C00E94A70608952091EF
:10126000FA0120FD02C021FF4CC080EE90E049C091
:101270008091FA0180FFF9CF89E390E042C080912C
:10128000FA0182FF0EC08091FA0184FF03C080E062
:1012900090E037C083EE90E034C08091FA0182FF85
:1012A000F2CF82EE90E02DC08091FA0183FF0BC057
:1012B0008091FA0184FDEBCF87EE90E022C080910F
:1012C000FA0183FFF5CF86EE90E01BC08091FA0112
:1012D00085FF07C089E290E014C08091FA0185FF84
:1012E000F9CF85E390E00DC08091FA0186FF07C039
:1012F0008AE290E006C08091FA0186FFF9CF81E38F
:1013000090E00E94B706089508950C948409809196
:101310006E010895CF93DF9300D01F92CDB7DEB753
:101320009C018091F101843019F593E099833B830E
:101330002A839093E9008FEF9091E800815095FD0A
:1013400006C095ED9A95F1F700008111F5CF8091D7
:10135000E80085FF0DC040E050E063E070E0CE01A2
:1013600001960E94F40B8091E8008E778093E8004C
:101370000F900F900F90DF91CF910895CF93DF934F
:1013800000D01F92CDB7DEB72091F101243021F5B6
:1013900022E029839B838A8383E08093E9008FEF97
:1013A0009091E800815095FD06C095ED9A95F1F772
:1013B00000008111F5CF8091E80085FF0DC040E06D
:1013C00050E063E070E0CE0101960E94F40B809142
:1013D000E8008E778093E8000F900F900F90DF91D8
:1013E000CF9108952091F1012430F1F422E020936F
:1013F000E9002FEF3091E800215035FD06C035EDB2
:101400003A95F1F700002111F5CF2091E80025FF72
:101410000BC040E050E065E070E00E94F40B80916A
:10142000E8008E778093E8000895CF93DF93EC0176
:101430009091F101943009F046C080910C0188230D
:10144000D9F080910D018823B9F09093E9008FEFD6
:101450009091E800815095FD06C095E19A95F1F7CD
:1014600000008111F5CF8091E80085FF2CC040E09D
:1014700050E060E170E017C081E08093E9008FEFF9
:101480009091E800815095FD06C095ED9A95F1F791
:1014900000008111F5CF8091E80085FF14C040E085
:1014A00050E068E070E0CE010E94F40B8091E8000B
:1014B0008E778093E80080E1FE01AEE5B1E0019017
:1014C0000D928A95E1F7DF91CF9108958091F00117
:1014D000811109C00E94890D0E94E60D8091E200F1
:1014E00084608093E20008951092F00108950895B9
:1014F0000C94CD220E942E1C0E94D3220E948C109C
:101500000C94850942E061EC81E00E94030D42E009
:1015100061EC82E00E94030D42E061EC83E00E94F6
:10152000030D42E161EC84E00C94030D8091F30122
:10153000833009F455C030F4813071F0823009F401
:101540008EC008958A3009F47AC08B3009F460C0E7
:10155000893009F09CC020C08091F201813A09F0E5
:1015600096C08091E800877F8093E8008091F60123
:101570009091F701892B21F460E18EE591E003C0A1
:1015800060E080E090E070E00E943F0C8091E80015
:101590008B778093E80008958091F201813209F001
:1015A00076C08091F6019091F701009719F00397AA
:1015B00009F06DC08091E800877F8093E8008091FA
:1015C000E80082FD05C08091F1018111F8CF5FC074
:1015D0008091F10080936E018091E8008B7753C079
:1015E0008091F201813A09F052C08091F601909108
:1015F000F701892B09F04BC08091E800877F809329
:10160000E8008091E80080FFFCCF80910C0136C09B
:101610008091F2018132D9F58091F6019091F70124
:10162000892BA9F58091E800877F8093E8000E94CC
:10163000380D8091F40180930C010C942515809154
:10164000F201813221F58091E800877F8093E800E4
:101650000E94380D8091F50180936F01089580916B
:10166000F201813AA1F48091E800877F8093E8003D
:101670008091E80080FFFCCF80916F018093F100A2
:101680008091E8008E778093E8000C94380D0895DF
:1016900084B7877F84BF88E10FB6F8948093600099
:1016A000109260000FBE90E080E80FB6F89480932F
:1016B0006100909361000FBE0E94DB100E94890DB3
:1016C0000E94E60D8091E20084608093E2007894AD
:1016D0000E946C100E94DD1082E091E00E94871051
:1016E0000E94BB228091F101853069F40E94F51BB4
:1016F0008091EF018823B1F30E94201C882391F38D
:101700000E94DE0BEFCF0E94E310ECCF292F33278E
:1017100023303105C9F064F42130310581F02230E5
:10172000310509F043C08DE690E022EE33E042C07F
:1017300021323105F1F02232310541F137C082E129
:1017400090E02FE434E036C099278130910541F0D4
:101750008230910541F0892B49F5EEEDF3E005C0AB
:10176000E6ECF3E002C0EEEAF3E0849190E09F0142
:1017700021C06430D8F4E62FF0E0EE0FFF1FEE5DDD
:10178000FE4F2081318189E090E014C0643070F414
:1017900070E0FB01EE0FFF1FE65EFE4F20813181FE
:1017A000FB01EA5EFE4F808190E004C080E090E0A3
:1017B00020E030E0FA0131832083089580E189BD83
:1017C00082E189BD09B400FEFDCF8091D8008F7DF4
:1017D0008093D8008091E00082608093E000809147
:1017E000E00081FDFCCF0895CF92DF92EF92FF924F
:1017F0000F931F93CF93DF93EC018B016A010E943B
:10180000570D811133C0C114D10439F0F601808124
:101810009181081B190BC80FD91FE12CF12C011560
:10182000110519F18091E80085FD16C08091E8004E
:101830008E778093E800C114D10449F0F6018081CD
:101840009181E80EF91EF182E08285E00FC00E94CE
:10185000570D882321F30AC089918093F10001502C
:101860001109FFEFEF1AFF0ADACF80E0DF91CF9185
:101870001F910F91FF90EF90DF90CF9008952091EE
:10188000F8013091F9012617370748F06115710505
:1018900039F42091E8002E772093E80001C0B901C7
:1018A00040E061157105A9F12091F101222309F4AD
:1018B00043C0253009F442C02091E80023FD40C018
:1018C0002091E80022FD32C02091E80020FFE9CFFE
:1018D0004091F3002091F20030E0342BFC01CF0165
:1018E0006115710559F02830310540F481918093DC
:1018F000F100615071092F5F3F4FF1CF41E0283077
:10190000310509F040E02091E8002E772093E800AF
:10191000C8CF4111C9CF0AC08091F101882361F07D
:10192000853061F08091E80083FD0AC08091E80075
:1019300082FFF2CF80E0089582E0089583E0089569
:1019400081E008952091F8013091F90126173707B9
:1019500048F06115710539F42091E8002E77209345
:10196000E80001C0B901FC0120E06115710591F1A9
:101970008091F101882309F440C0853009F43FC00B
:101980008091E80083FD3DC08091E80082FD2FC07A
:101990008091E80080FFE9CF2091F3008091F20070
:1019A00090E0922B6115710559F08830910540F453
:1019B00024912093F1003196615071090196F2CF84
:1019C00021E0089709F020E08091E8008E7780936D
:1019D000E800CBCF2111CCCF0AC08091F101882340
:1019E00061F0853061F08091E80083FD0AC080914C
:1019F000E80082FFF2CF80E0089582E0089583E05E
:101A0000089581E00895982F973058F59093E90054
:101A1000981739F07091EC002091ED005091F00092
:101A200003C0242F762F50E021FF19C03091EB0026
:101A30003E7F3093EB003091ED003D7F3093ED0021
:101A40003091EB0031603093EB007093EC00209309
:101A5000ED005093F0002091EE0027FF07C09F5F3C
:101A6000D3CF8F708093E90081E0089580E00895DE
:101A70008091F20187FF11C08091E80082FD05C0CE
:101A80008091F1018111F8CF11C08091E8008B772E
:101A90000BC08091F101882349F08091E80080FF1C
:101AA000F8CF8091E8008E778093E8000895209128
:101AB000E4003091E50095E64091EC00842F8170C0
:101AC00040FF22C08091E80080FD1CC08091F101A0
:101AD000882391F0853091F08091EB0085FD10C056
:101AE0004091E4005091E5004217530729F39A0111
:101AF000915011F784E0089582E0089583E00895FD
:101B000081E0089580E008954091E80042FFDECF33
:101B100008950E94F70D0E94FF0DE0EEF0E0808135
:101B200081608083E8EDF0E080818F77808319BC4D
:101B3000A7EDB0E08C918E7F8C9380818F7E808327
:101B40001092F00108950F931F93CF93DF930E949B
:101B5000F70D0E94FF0DC8EDD0E088818F77888354
:101B600088818068888388818F7D888319BC1092E2
:101B7000F1011092ED011092EF011092EE0100EED2
:101B800010E0F80180818B7F808388818160888369
:101B900042E060E080E00E94030DE1EEF0E0808131
:101BA0008E7F8083E2EEF0E080818160808380819F
:101BB00088608083F80180818E7F80838881806146
:101BC0008883DF91CF911F910F910895E8EDF0E0A8
:101BD00080818F7E8083E7EDF0E08081816080836B
:101BE00084E082BF81E08093F0010C94A30DE8EDC6
:101BF000F0E080818E7F80831092E2000895109241
:101C0000DA001092E10008951F920F920FB60F9222
:101C100011242F933F934F935F936F937F938F93F1
:101C20009F93AF93BF93EF93FF938091E10082FF67
:101C30000BC08091E20082FF07C08091E1008B7FA2
:101C40008093E1000E946B108091DA0080FF1FC03A
:101C50008091D80080FF1BC08091DA008E7F809336
:101C6000DA008091D90080FF0DC080E189BD82E15A
:101C700089BD09B400FEFDCF81E08093F1010E948F
:101C8000660A05C019BC1092F1010E94740A809185
:101C9000E10080FF19C08091E20080FF15C08091B3
:101CA000E2008E7F8093E2008091E2008061809369
:101CB000E2008091D80080628093D80019BC85E052
:101CC0008093F1010E94780A8091E10084FF30C086
:101CD0008091E20084FF2CC080E189BD82E189BD52
:101CE00009B400FEFDCF8091D8008F7D8093D8008D
:101CF0008091E1008F7E8093E1008091E2008F7EF1
:101D00008093E2008091E20081608093E200809104
:101D1000ED01882311F084E007C08091E30087FD86
:101D200002C081E001C083E08093F1010E947A0A41
:101D30008091E10083FF29C08091E20083FF25C0EC
:101D40008091E100877F8093E10082E08093F10140
:101D50001092ED018091E1008E7F8093E1008091EF
:101D6000E2008E7F8093E2008091E20080618093A8
:101D7000E20042E060E080E00E94030D8091F0000C
:101D800088608093F0000E94770AFF91EF91BF91E5
:101D9000AF919F918F917F916F915F914F913F9103
:101DA0002F910F900FBE0F901F9018951F920F92BA
:101DB0000FB60F9211242F933F934F935F936F931E
:101DC0007F938F939F93AF93BF93CF93DF93EF93C3
:101DD000FF93C091E900CF708091EC00D82FD170B3
:101DE00080FDD0E81092E9008091F000877F809319
:101DF000F00078940E941A0F1092E9008091F00090
:101E000088608093F000CD2BCF70C093E900FF91E4
:101E1000EF91DF91CF91BF91AF919F918F917F9182
:101E20006F915F914F913F912F910F900FBE0F9047
:101E30001F9018951F93CF93DF93CDB7DEB7AA9766
:101E40000FB6F894DEBF0FBECDBFE2EFF1E088E041
:101E50008E0F9091F10091938E13FBCF0E94960A02
:101E60008091E80083FF1FC18091F2019091F301FE
:101E7000492F50E04A30510508F015C1FA01EA5ADD
:101E8000FF4F0C945524803881F0823809F00BC143
:101E90008091F6018F708093E9008091EB0085FBC3
:101EA000882780F91092E90006C08091EE01909198
:101EB000EF01911182609091E800977F9093E80084
:101EC0008093F1001092F100C8C0282F2D7F09F0F7
:101ED000EAC0882319F0823061F0E5C08091F401F6
:101EE000813009F0E0C0933009F080E08093EF0189
:101EF0002BC08091F401811127C08091F6018F7071
:101F000009F4D1C08093E9002091EB0020FF1CC0B0
:101F1000933021F48091EB00806214C09091EB002B
:101F200090619093EB0021E030E0A90102C0440FE2
:101F3000551F8A95E2F74093EA001092EA008091DB
:101F4000EB0088608093EB001092E9008091E8003C
:101F5000877F86C08111A7C01091F4011F778091FF
:101F6000E3008078812B8093E3008091E800877FF5
:101F70008093E8000E94380D8091E80080FFFCCF3C
:101F80008091E30080688093E300111102C082E039
:101F900001C083E08093F10186C08058823008F050
:101FA00082C08091F4019091F5018C3D53E095073A
:101FB00079F583E08A838AE289834FB7F894DE015A
:101FC000139620E03EE051E2E32FF0E050935700FB
:101FD000E49120FF03C0E295EF703F5FEF708E2F1A
:101FE00090E0EA3010F0C79601C0C0968D939D93A3
:101FF0002F5F243149F74FBF8091E800877F80939E
:10200000E8006AE270E0CE0101960E943F0C14C025
:10201000AE014F5F5F4F6091F6010E94860BBC01DD
:10202000009709F440C09091E800977F9093E800F2
:1020300089819A810E94A20C8091E8008B7780931D
:10204000E80031C0803879F58091E800877F80937F
:10205000E8008091ED018093F1008091E8008E7797
:102060008093E8000E94380D1EC081111CC0909121
:10207000F4019230C0F48091E800877F8093E800FB
:102080009093ED010E94380D8091ED01811106C001
:102090008091E30087FD02C081E001C084E080936D
:1020A000F1010E94820A8091E80083FF0AC08091BA
:1020B000E800877F8093E8008091EB008062809346
:1020C000EB00AA960FB6F894DEBF0FBECDBFDF912E
:1020D000CF911F9108950895CF938091F1018823A6
:1020E000A1F0C091E900CF709091EC00892F817030
:1020F00090FD80E8C82B1092E9008091E80083FDF4
:102100000E941A0FCF70C093E900CF910895909369
:102110007501809374010895E0917401F091750147
:10212000309721F00190F081E02D099480E008952E
:10213000E0917401F0917501309721F00280F381F4
:10214000E02D09940895E0917401F09175013097A4
:1021500021F00480F581E02D099408952091720109
:10216000309173018217930771F0909373018093FC
:102170007201E0917401F0917501309721F00680B1
:10218000F781E02D0994089520917001309171013B
:102190008217930771F09093710180937001E09121
:1021A0007401F0917501309721F00084F185E02DE4
:1021B0000994089508950C94DA100E94341C0E942A
:1021C00087030C94F61C9F92AF92BF92CF92DF923E
:1021D000EF92FF920F931F93CF93DF9300D000D025
:1021E00000D0CDB7DEB70E949F030DE010E0AA2417
:1021F000A394B12C902E802F0E948D049801295811
:102200003E4F6901F901F080F826A1F4015011094F
:1022100088F78FEF89838A831B820E943D1C81602F
:10222000782F9D838C8349815A816B818D810E9497
:102230007A112FC09091DA0191FF04C08E830E9421
:1022400093048E8125E030E0A501022E01C0440FE9
:102250000A94EAF7E42E4F21C1F029839A828E2155
:1022600091E009F490E09B830E943D1C8160782FEF
:102270009D838C8349815A816B818D810E947A1163
:10228000F6018081E826E08204C021503109E0F6A1
:10229000BDCF0E94DD1F109176010E948C1018178F
:1022A000B9F00E948C108093760126960FB6F894B0
:1022B000DEBF0FBECDBFDF91CF911F910F91FF9079
:1022C000EF90DF90CF90BF90AF909F900C948509D6
:1022D00026960FB6F894DEBF0FBECDBFDF91CF912B
:1022E0001F910F91FF90EF90DF90CF90BF90AF9034
:1022F0009F900895CF93DF93CDB7DEB72B970FB69E
:10230000F894DEBF0FBECDBF4F83588769877A87A9
:102310008B87DE01119686E0FD0111928A95E9F71F
:1023200085E0FE01379601900D928A95E1F749818B
:102330005A816B817C818D819E810E94C3172B966F
:102340000FB6F894DEBF0FBECDBFDF91CF910895D9
:10235000CF93882309F4C2C0C82F823859F40E9451
:102360008C1081FDBBC089E30E949D1A0E946A1BEC
:1023700089E30CC0833879F40E948C1080FDAEC0D4
:1023800083E50E949D1A0E946A1B83E50E94DF1A62
:10239000CF910C946A1B843859F40E948C1082FDF2
:1023A0009DC087E40E949D1A0E946A1B87E4EECFBD
:1023B0008CEF8C0F813A48F48C2F0E9420228111DF
:1023C0008DC08C2F0E949D1AE3CF80E28C0F883045
:1023D00048F4C77081E001C0880FCA95EAF70E94EF
:1023E000231BD6CF8BE58C0F833078F4C53A29F0C8
:1023F000C63A31F083E890E005C081E890E002C081
:1024000082E890E0CF910C94AE1088E58C0F833178
:1024100008F064C0C83A39F1C93A41F1CA3A49F101
:10242000CB3A51F1CC3A59F1CD3A61F1C03B69F167
:10243000CE3A71F1CF3A79F1C13B81F1C23B89F1DA
:10244000C33B91F1C43B99F1C53BA1F1C63BA9F156
:10245000C73BB1F1C83BB9F1C93BC1F1CA3BC9F1B6
:1024600080E090E038C082EE90E035C089EE90E0E8
:1024700032C08AEE90E02FC085EB90E02CC086EB56
:1024800090E029C087EB90E026C08CEC90E023C060
:102490008DEC90E020C083E891E01DC08AE891E0D7
:1024A0001AC082E991E017C084E991E014C081E28A
:1024B00092E011C083E292E00EC084E292E00BC091
:1024C00085E292E008C086E292E005C087E292E0F1
:1024D00002C08AE292E0CF910C94C410CF9108958B
:1024E000882309F44BC0823859F40E948C1081FF74
:1024F00045C089E30E949D1A0E946A1B89E30CC0B3
:10250000833871F40E948C1080FF38C083E50E94EC
:102510009D1A0E946A1B83E50E94DF1A0C946A1BB5
:10252000843859F40E948C1082FF28C087E40E94EE
:102530009D1A0E946A1B87E4EFCF9CEF980F913A97
:1025400058F390E2980F983050F4877091E001C0F2
:10255000990F8A95EAF7892F0E94291BDFCF9BE507
:10256000980F933020F480E090E00C94AE10885ADD
:10257000833120F480E090E00C94C4100895882307
:1025800021F00E94231B0C946A1B0895882321F0DC
:102590000E94291B0C946A1B08957F928F929F9230
:1025A000AF92BF92CF92DF92EF92FF920F931F9361
:1025B000CF93DF931F92CDB7DEB77C01C62E772E67
:1025C000FC01058102950F70128111110E94401BC0
:1025D0000E94961A882379F0112369F080E28C0D0D
:1025E000883048F082E00E947F1A0E94961A91E09B
:1025F000D82ED92601C0D12CE72DE295EF70F0E05E
:10260000E05AFF4F0C945524872D807F072D0F70C3
:10261000882311F00295007F112389F0002309F42B
:1026200090C180E28C0D883020F4802F0E94231B03
:1026300003C0802F0E94331B0E946A1B82C18C2D15
:102640000E947012002309F495C180E28C0D88303D
:1026500020F4802F0E94291B03C0802F0E94391B69
:102660000E946A1B87C1972D907F872D8F709032B3
:1026700011F08295807FCC2021F0F1E0CF16B1F0EF
:102680001EC0112349F0002309F414C1013009F0E0
:1026900011C10E94531B6EC1002319F0013009F4CF
:1026A00069C189830E94561B89810AC1112321F0C7
:1026B000023008F05FC1FEC001115CC101C11123ED
:1026C00021F0002309F4F6C03CC1002309F4F8C04E
:1026D0003EC1872D86958695837090E0009719F00E
:1026E000019761F047C1112321F08C2D972D937034
:1026F00002C080E090E00E94AE103CC1112321F0A6
:102700008C2D972D937002C080E090E00E94C41041
:1027100031C18C2D112319F00E94E51E02C00E94C8
:102720004D1F0E94D21F26C1872D837009F052C011
:10273000111120C18C2D829586958770880F880F86
:102740009C2D9F70892E912CA12CB12C082E04C099
:10275000880C991CAA1CBB1C0A94D2F7C4FE14C096
:102760000FE010E020E030E0B901A80104C0440F00
:10277000551F661F771F8A95D2F7CB01BA01609566
:1027800070958095909503C060E070E0CB01272D97
:1027900026952695237030E02230310569F02330EC
:1027A000310589F0682979298A299B292130310549
:1027B00071F00E940B19DEC0682979298A299B29AA
:1027C0000E942719D7C00E940B19C501B4010E94AD
:1027D000EF18D0C0112319F0872D817001C08695A4
:1027E000882309F4C7C08C2D829586958770880F41
:1027F000880F9C2D9F70892E912CA12CB12C082E16
:1028000004C0880C991CAA1CBB1C0A94D2F7C4FEF5
:1028100014C00FE010E020E030E0B901A80104C0CE
:10282000440F551F661F771F8A95D2F7CB01BA0157
:10283000609570958095909503C060E070E0CB0145
:10284000272D269526952370422F50E042305105C2
:1028500069F04330510589F0682979298A299B2933
:102860004130510571F00E94E51984C06829792929
:102870008A299B290E94011A7DC00E94E519C50181
:10288000B4010E94C91976C08C2D90E0FC01E05E75
:10289000F109E531F10508F050C0E059FF4F0C9403
:1028A00055240C2D0F70872D8F71112331F00E944C
:1028B0006219802F0E94BF125DC00E948319802F71
:1028C0000E94C61257C0112339F0011153C0872D41
:1028D0008F710E94A8194EC0023008F04BC0F7CF8C
:1028E000112339F0872D8F710E94621943C0112383
:1028F000C9F3872D8F710E9483193CC0112329F0E1
:10290000872D8F710E944D1935C00E94431932C026
:10291000112351F0172D1F71812F0E94621963E05E
:10292000812F0E94761A26C081E00E947F1A023011
:1029300008F182E00E947F1A1DC0112331F00023AC
:1029400089F28C2D0E94A81115C0002391F28C2DC4
:102950000E9470120FC0472D4F706C2DC7010E944E
:10296000A9050E94671806C0472D4F706C2DC7013E
:102970000E949406DD20F9F00E94721A80FD1BC0AF
:10298000F70112820E946C1A0E946219C7010E940C
:10299000EA140E946C1A0F90DF91CF911F910F9152
:1029A000FF90EF90DF90CF90BF90AF909F908F906F
:1029B0007F900C9483190F90DF91CF911F910F910D
:1029C000FF90EF90DF90CF90BF90AF909F908F904F
:1029D0007F9008950F931F93CF93DF93EC0188812D
:1029E00099812B813C81232BB9F09F3F11F48F3FBC
:1029F00099F0CE010E94EC05882371F068817981FD
:102A00008A810E94681A8C010E941D1A0E94E41893
:102A1000B801CE010E94CD12DF91CF911F910F918D
:102A200008950E94401B0E94501B0E94151B0E948B
:102A30006A1B0E9483200E94D21F80E090E00E94C7
:102A4000AE1080E090E00C94C4100E94301B0C94F7
:102A500011150E945D1A292F22952F7030E02C301D
:102A600031054CF42A3031056CF422503109223002
:102A70003105A8F407C02C30310569F02F3031053D
:102A800051F00DC0803F69F018F4803E40F409C059
:102A9000843F29F406C093FB882780F9089580E0DD
:102AA000089581E00895CF93DF9300D000D01F9266
:102AB000CDB7DEB70F900F900F900F900F90DF9172
:102AC000CF910895CF93DF9300D000D000D0CDB741
:102AD000DEB726960FB6F894DEBF0FBECDBFDF91EE
:102AE000CF9108951F93CF93DF93C091850116E096
:102AF00080918601C81799F0D0E01C9FF0011D9FBE
:102B0000F00D1124E957FE4F40815181628173819C
:102B1000848195810E9462152196C770E9CFDF916B
:102B2000CF911F9108954091B7015091B8016091E4
:102B3000B9017091BA018091BB019091BC010C94D4
:102B400062158091BC0182958F7009F054C080910C
:102B5000B901882309F44FC080918501A0918601B5
:102B60006091B7017091B8014091BA015091BB01D9
:102B7000B6E08A1709F43FC090E041155105C1F154
:102B80007F3F11F46F3FA1F1B89FF001B99FF00DA5
:102B90001124E957FE4F218172132AC0208162134C
:102BA00027C02281211124C02381348124173507B5
:102BB00010F421503109241B350B283C3105C0F499
:102BC0002091BC012F7020612093BC0126E0289F3A
:102BD000F001299FF00D1124E457FE4F80818F7082
:102BE0008061808387EB91E00E94EA140C94721557
:102BF00001968770BECF0895CF92DF92EF92FF9239
:102C00000F931F93CF93DF93CDB7DEB762970FB6C5
:102C1000F894DEBF0FBECDBF8C0185E0F801DE0168
:102C20001D9601900D928A95E1F7D8014C9111966D
:102C30005C91119712966C9112971396CD90DC903F
:102C400014973091B7017091B8018091BA019091B9
:102C5000BB01009709F46BC17F3F19F43F3F09F4B2
:102C600066C1E090B901EE2009F4C0C02091BC011A
:102C7000C816D90628F0F601E81BF90BCF0104C0ED
:102C8000809590958C0D9D1DFF24F394883C9105B3
:102C900078F0F12C207F09F0C6C07C2DD98AC88A33
:102CA00089890E94531587EB91E00E94EA14B1C014
:102CB000822F807F09F046C0751314C0341312C0F0
:102CC000611110C02F7020612093BC010E949315E8
:102CD00087EB91E00E94EA148091BC01D80115961F
:102CE0008C932EC0CD2819F15F3F11F44F3FF9F0BE
:102CF000F62E61111CC0809185012091860136E07D
:102D0000821709F45AC090E0389FF001399FF00D06
:102D10001124E957FE4F7181571306C07081471384
:102D200003C07281711103C001968770E9CFF62E3E
:102D3000662309F418C18091BC0181608093BC01B5
:102D4000F12C11C1751308C0341306C0611104C001
:102D50008091BC01D801C3C04D875E878D859E855B
:102D60006A8B0E9429156A898823E1F16623D1F1D3
:102D70002091BC01822F82958F7090E0029774F0B1
:102D80008091B7019091B80198878F831986DB866F
:102D9000CA862C87CE0107960E94EA1486E0F801C5
:102DA000A7EBB1E001900D928A95E1F70E94A11581
:102DB0000E949315FF24F394D6C04D875E878D85BE
:102DC0009E850E945D1A292F22952F7030E02230B7
:102DD00031050CF0BCC09F7009F0B6C0805E883031
:102DE00008F4C1C0C8010E94EA14E4CFC816D9068D
:102DF00008F453C0F601E81BF90BCF01883C91059C
:102E000008F450C0F12C7C2DD98AC88A89890E9487
:102E10005315E7EBF1E086E0DF011D928A95E9F7B3
:102E20000E949315A0C0751314C0341312C0611111
:102E300010C08091BC01F8018583C8010E94EA148A
:102E400086E0E7EBF1E0DF011D928A95E9F7FE2CC1
:102E50008AC04D875E878D859E856A8B0E94291565
:102E60006A89882309F4BECF662309F4BBCF209179
:102E7000BC01822F82958F7090E002970CF48ECF68
:102E80008091B7019091B8019A8389831B82DD827A
:102E9000CC822E83CE0101967FCF809590958C0DAC
:102EA0009D1DACCFF62E662309F49CCF75132EC062
:102EB00034132CC02091BC0120FD1FC0822F8295AD
:102EC0008F70D9F0D80115962C9315978F3049F053
:102ED0008F5F982F9295907F822F8F70892B1596F8
:102EE0008C93C8010E94EA1486E0F801A7EBB1E0D8
:102EF00001900D928A95E1F793CF86E0F801A7EB58
:102F0000B1E001900D928A95E1F72DC04D875E8763
:102F10008D859E850E942915811140CF8091BC012D
:102F200081608093BC01C8010E94EA141CC0662322
:102F300009F458CF4D875E878D859E850E9429159F
:102F4000882309F44FCF2ACF811148CF0CC02430F9
:102F500031050CF047CF9F7009F440CFF8019581FF
:102F6000907F09F03BCF8F2D62960FB6F894DEBFAD
:102F70000FBECDBFDF91CF911F910F91FF90EF90CA
:102F8000DF90CF9008951F93CF93DF93CDB7DEB737
:102F90002C970FB6F894DEBF0FBECDBF4F83588776
:102FA00069877A878B879C87CE0107960E94FC15DC
:102FB000882369F08F8198852A853B85232BF1F141
:102FC0009F3F09F063C08F3F09F060C037C086E0C3
:102FD000FE013796DE01119601900D928A95E1F778
:102FE0006F817885EA85FB85309741F17F3F11F449
:102FF0006F3F21F12091860130E0C9010196877071
:1030000099274091850150E08417950709F447C03E
:1030100069837A83FD83EC8396E0929FD001939F2E
:10302000B00D1124A957BE4FFE01319601900D92AB
:103030009A95E1F7809386010E94721516E08091BF
:103040008501909186018917C1F1189FC001112453
:1030500089579E4F0E94FC15882379F1E0918501E4
:103060001E9FF0011124E957FE4F4081518162817A
:103070007381848195810E9462158091850190E021
:1030800001968770992780938501D9CF4F81588504
:1030900069857A858B859C850E946215CFCF0E94B9
:1030A00025151092860110928501E7EBF1E086E08C
:1030B000DF011D928A95E9F7C1CF2C960FB6F894DF
:1030C000DEBF0FBECDBFDF91CF911F910895EF926C
:1030D000FF920F931F93CF93DF938C01009709F416
:1030E0006CC0F12CEE24E394E8012196F801849160
:1030F000843740F4843008F051C0813081F0823050
:1031000019F15BC0853709F444C0A8F19CE7980F1A
:10311000903708F052C08F770E94701241C00E5F46
:103120001F4FFE01C49180E28C0F883048F4C770B5
:103130008E2D01C0880FCA95EAF70E94431B14C068
:103140008C2F0E94A8112DC00E5F1F4FFE01C4914D
:1031500080E28C0F883058F4C7708E2D01C0880F24
:10316000CA95EAF70E94491B0E946A1B1AC08C2F5D
:103170000E94701216C00E5F1F4FFE01C491CC2337
:1031800081F08FE99FE00197F1F700C00000C15086
:10319000F6CF0E5F1F4FFE01F49003C00E94A811EE
:1031A0008E018F2D882309F49FCFEFE9FFE031973F
:1031B000F1F700C000008150F5CFDF91CF911F9152
:1031C0000F91FF90EF90089508956093C10170935F
:1031D000C2018093C3019093C4010C9411150F9305
:1031E0001F930091C1011091C2012091C301309140
:1031F000C401DC01CB01802B912BA22BB32B80933C
:10320000C1019093C201A093C301B093C4011F9167
:103210000F910C9411150F931F930091C101109100
:10322000C2012091C3013091C401DC01CB01802394
:103230009123A223B3238093C1019093C201A09351
:10324000C301B093C4011F910F910C9411150F93FA
:103250001F930091C1011091C2012091C3013091CF
:10326000C401DC01CB0180279127A227B3278093DB
:10327000C1019093C201A093C301B093C4011F91F7
:103280000F910C9411151092BD011092BE01109275
:10329000BF011092C0010C94111541E050E060E0B4
:1032A00070E004C0440F551F661F771F8A95D2F740
:1032B0004093BD015093BE016093BF017093C00164
:1032C0000C94111541E050E060E070E004C0440F40
:1032D000551F661F771F8A95D2F78091BD01909187
:1032E000BE01A091BF01B091C001482B592B6A2BA0
:1032F0007B2B4093BD015093BE016093BF0170933F
:10330000C0010C94111541E050E060E070E004C091
:10331000440F551F661F771F8A95D2F74095509529
:10332000609570958091BD019091BE01A091BF0103
:10333000B091C001482359236A237B234093BD01E8
:103340005093BE016093BF017093C0010C9411159E
:1033500041E050E060E070E004C0440F551F661F7C
:10336000771F8A95D2F78091BD019091BE01A091FF
:10337000BF01B091C001482759276A277B27409396
:10338000BD015093BE016093BF017093C0010C94C6
:1033900011150F931F930091BD011091BE01209153
:1033A000BF013091C001DC01CB01802B912BA22BFE
:1033B000B32B8093BD019093BE01A093BF01B09346
:1033C000C0011F910F910C9411150F931F93009141
:1033D000BD011091BE012091BF013091C001DC01FF
:1033E000CB0180239123A223B3238093BD0190932B
:1033F000BE01A093BF01B093C0011F910F910C9427
:1034000011150F931F930091BD011091BE012091E2
:10341000BF013091C001DC01CB0180279127A22799
:10342000B3278093BD019093BE01A093BF01B093D9
:10343000C0011F910F910C9411150895CF92DF9246
:10344000EF92FF920F931F93CF93DF938C01C09065
:10345000C101D090C201E090C301F090C4018091FD
:10346000BD019091BE01A091BF01B091C001C82AD9
:10347000D92AEA2AFB2ACFE1D0E0D701C6010C2ED7
:1034800004C0B695A795979587950A94D2F780FFC3
:1034900006C0B8018C2F0E94EA08019721F42197F9
:1034A00060F780E001C08C2FDF91CF911F910F91C9
:1034B000FF90EF90DF90CF900895CF93DF93EC01D2
:1034C0000E941E1ABE010E94EA08DF91CF91089562
:1034D000CB010E945D1A08958091C501859585955F
:1034E000859508958091C5018770089598E0899F1A
:1034F00090011124262B2093C5010C946219209170
:10350000C501809582238093C501982F977069F437
:1035100030E0482F552747FD50952417350729F0EF
:103520008595859585950C94831908959091C5018D
:10353000977081E009F480E0089590910C0199233F
:1035400021F090910D01911109C020910E0130914F
:103550000F01F90132969FEF40E01FC0982F96951A
:10356000969596959F3050F5E0910E01F0910F01E0
:10357000E90FF11D877021E030E0A90102C0440F7E
:10358000551F8A95E2F7CA019181892B818308959D
:103590009F3F39F04F5F4E3041F051915813F8CFB3
:1035A0000DC05111F7CF942FF5CF9F3F39F0F9019E
:1035B000E90FF11D97FDFA95828308950895909182
:1035C0000C01992321F090910D01911109C02091D6
:1035D0000E0130910F01F9013296205F3F4F1FC05D
:1035E000982F9695969596959F30F0F4E0910E0160
:1035F000F0910F01E90FF11D877021E030E0A90182
:1036000002C0440F551F8A95E2F7CA018095918147
:103610008923818308953196E217F30729F0908179
:103620009813F9CF1082F7CF089581E090E0E091F0
:103630000E01F0910F01E80FF91F10820196803101
:103640009105A9F708959091D901892B8093D9010B
:10365000089580959091D90189238093D901089587
:103660001092D90108959091D801892B8093D801A7
:10367000089580959091D80189238093D801089569
:103680001092D80108959091D701892B8093D7018A
:10369000089580959091D70189238093D70108954B
:1036A0001092D70108958093C60108951092C60123
:1036B000089580910E0190910F01FC0131969C01BB
:1036C000205F3F4F80E0919191118F5FE217F307E8
:1036D000D1F70895E0910E01F0910F018091D90189
:1036E0008083E0910E01F0910F0190818091D801CB
:1036F000892B8083E0910E01F0910F0190818091E0
:10370000D701892B80838091C601882361F0E091E5
:103710000E01F0910F019081892B80830E94591B2B
:1037200081111092C60180910E0190910F010C94AD
:10373000981020E0009739F0AC01415051098423E2
:1037400095232F5FF7CF822F0895CF92DF92EF92CC
:10375000FF926C01EE24FF24C114D104E104F104B2
:1037600021F0C701B60120E101C020E0C72ED82E0C
:10377000E92EFF24C114D104E104F10419F0285FFB
:10378000C701B6016B017C0154E0F694E794D7942D
:10379000C7945A95D1F7C114D104E104F10419F08A
:1037A0002C5FC701B6016B017C0142E0F694E794FF
:1037B000D794C7944A95D1F7C114D104E104F10418
:1037C00019F02E5FC701B601DC01CB01B695A795B4
:1037D00097958795892B8A2B8B2B09F02F5F822F4A
:1037E000FF90EF90DF90CF9008958091F1018430A9
:1037F00021F11092DB0120E488E190E00FB6F8940B
:10380000A895809360000FBE2093600080E00E9426
:10381000850983B7817F846083BF83B7816083BF5D
:103820007894889583B78E7F83BF88E10FB6F8942C
:1038300080936000109260000FBE0895089508956F
:103840000E941E1C0E949F030E941F1C0E94940441
:1038500091E0811101C090E0892F08950E94251503
:103860000E948C100C94850982E084BD93E095BD84
:103870009AEF97BD80936E0008952FB7F8948091CA
:10388000DC019091DD01A091DE01B091DF012FBF3D
:103890000895CF92DF92EF92FF920F931F932FB76D
:1038A000F8944091DC015091DD016091DE0170914E
:1038B000DF012FBF6A017B01EE24FF248C0120E091
:1038C00030E0C016D106E206F30610F4415051096B
:1038D0009A01281B390BC9011F910F91FF90EF909E
:1038E000DF90CF9008951F920F920FB60F92112480
:1038F0008F939F93AF93BF938091DC019091DD01F3
:10390000A091DE01B091DF010196A11DB11D809350
:10391000DC019093DD01A093DE01B093DF01BF9144
:10392000AF919F918F910F900FBE0F901F901895A0
:103930000E94890DF8942FEF87EA91E6215080408C
:103940009040E1F700C0000087E090EBDC0180933D
:10395000FB019093FC01A093FD01B093FE019CE05C
:1039600088E10FB6F894A895809360000FBE9093FD
:103970006000FFCFEF92FF920F931F93CF93DF93DF
:10398000D82FCDE08C2F0E948D0405E010E0E82EAA
:10399000F12CC701002E02C0959587950A94E2F795
:1039A00080FF09C0602F7C2F80E00E949506D8130D
:1039B00002C081E006C00150110958F7C15010F74C
:1039C00080E0DF91CF911F910F91FF90EF900895CC
:1039D000CF93C82F8CE20E94BA1C882321F08C2F31
:1039E000CF910C94BA1C80E0CF910895CF930E94A0
:1039F0003D1E811102C00E94231EC5E6C15049F040
:103A00000E949F038FE39CE90197F1F700C000003B
:103A1000F5CF89E20E94E81C811113C18AE20E945D
:103A2000E81C81110E94231E85E00E94E81C811180
:103A30000E94981C0E94481E8093DA0187E00E9431
:103A4000E81C8823A9F18BE10E94E81C882351F02F
:103A50008091DA0181FB222720F991E0922790FBE7
:103A600081F90EC08EE00E94E81C882361F08091ED
:103A7000DA0182FB222720F991E0922790FB82F95C
:103A80008093DA0115C080E10E94E81C9091DA0170
:103A9000882341F093FB222720F981E0822780FBD5
:103AA00093F904C0892F809580FB90F99093DA01F7
:103AB0008091DA010E944C1E0E945A1E8093FA01E6
:103AC00080EE0E94E81C882341F08091FA01982F33
:103AD000909590FB80F98093FA0189E30E94E81C9D
:103AE000882359F08091FA0181FB222720F991E087
:103AF000922790FB81F98093FA0182EE0E94E81CE4
:103B0000882359F08091FA0182FB222720F991E065
:103B1000922790FB82F98093FA0186EE0E94E81CBE
:103B2000882359F08091FA0183FB222720F991E044
:103B3000922790FB83F98093FA0183EE0E94E81CA0
:103B4000882359F08091FA0184FB222720F991E023
:103B5000922790FB84F98093FA0185E30E94E81C88
:103B6000882359F08091FA0185FB222720F991E002
:103B7000922790FB85F98093FA0181E30E94E81C6B
:103B8000882359F08091FA0186FB222720F991E0E1
:103B9000922790FB86F98093FA0181E10E94E81C4C
:103BA000882359F08091FA0187FB222720F991E0C0
:103BB000922790FB87F98093FA018091FA010E9485
:103BC0005E1E8091FA0187FB882780F980930D01A2
:103BD00087E20E94E81CC82F8EE10E94E81C811138
:103BE000C2608FE10E94E81C8111C46080E20E94E3
:103BF000E81C8111C86081E20E94E81C8111C0614B
:103C000082E20E94E81C8111C06283E20E94E81CEB
:103C10008111C06484E20E94E81C882311F0C0680E
:103C200002C0CC2329F08C2F0E94551E6C2F03C09C
:103C30000E94511E682F70E080E090E0CF910C94BC
:103C4000E518CF9108956DEE7EEF80E090E00E9440
:103C50008F2460E082E090E00E947D2460E083E0B9
:103C600090E00E947D2460E084E090E00E947D244A
:103C700060E085E090E00C947D2480E090E00E947C
:103C8000772421E08D3E9E4F09F020E0822F089599
:103C900082E090E00C946F24682F82E090E00C9416
:103CA0007D2483E090E00C946F24682F83E090E003
:103CB0000C947D2484E090E00C946F24682F84E0C1
:103CC00090E00C947D248091E20180FF0BC0609114
:103CD000130185E0689FB00111247595679575956E
:103CE00067952BC081FF09C06091130185E0689F33
:103CF000B00111247595679520C082FF07C06091BF
:103D0000130185E0689FB001112417C09091E30171
:103D10009923D1F060911201961788F72091130131
:103D200085E0289F90011124929FA001939F500D40
:103D3000112470E0CA010E9441246038710540F4EA
:103D40006115710539F002C065E070E0862F0895B5
:103D50008FE7089581E008958091E20180FF08C017
:103D60006091110170E0759567957595679521C013
:103D700081FF06C06091110170E07595679519C0CB
:103D800082FF04C06091110170E010C09091E301C6
:103D90009923C1F0609110019617A0F7809111014D
:103DA000899FC001112470E00E9441246038710590
:103DB00028F46115710521F0862F08958FE7089585
:103DC00081E0089561E070E0F4CF803F21F40E942B
:103DD000631E819504C0813F29F40E94631E809375
:103DE000E6010895823F21F40E94631E819504C07C
:103DF000833F29F40E94631E8093E5010895893F63
:103E000019F40E94AC1E05C08A3F31F40E94AC1E1A
:103E100081958093E70108958B3F21F40E94AC1EA9
:103E2000819504C08C3F29F40E94AC1E8093E80168
:103E30000895843F21F48091E401816017C0853F9B
:103E400021F48091E401826011C0863F21F48091C9
:103E5000E40184600BC0873F21F48091E401886015
:103E600005C0883F31F48091E40180618093E401D2
:103E700008958D3F21F48091E20181600BC08E3F57
:103E800021F48091E201826005C08F3F29F4809186
:103E9000E20184608093E2010895803F39F48091CB
:103EA000E60187FF6CC01092E60169C0813F29F4EA
:103EB0008091E6011816BCF362C09091E501823F43
:103EC00029F497FF5CC01092E50159C0833F19F4B3
:103ED0001916CCF354C0893F41F48091E7011816BC
:103EE0000CF04DC01092E7014AC08A3F29F480913E
:103EF000E70187FF44C0F6CF8B3F39F48091E8019A
:103F000087FF3DC01092E8013AC08C3F29F48091B0
:103F1000E8011816BCF333C0843F21F48091E4011A
:103F20008E7F17C0853F21F48091E4018D7F11C001
:103F3000863F21F48091E4018B7F0BC0873F21F401
:103F40008091E401877F05C0883F31F48091E401CE
:103F50008F7E8093E40113C08D3F21F48091E201B4
:103F60008E7F0BC08E3F21F48091E2018D7F05C0D2
:103F70008F3F29F48091E2018B7F8093E201809151
:103F8000E50181110EC08091E60181110AC0809186
:103F9000E701811106C08091E801811102C01092F1
:103FA000E301089584EE91E00E94A3100E943D1C5D
:103FB0009093E1018093E00108951F93CF93DF93E5
:103FC0008091E0019091E1010E94491CAC01909127
:103FD000E301992321F02091140130E006C02091E3
:103FE00015018AE0289F900111244217530708F415
:103FF00086C08091E501C091E601D091E701109162
:10400000E801811107C0C11176C0D11174C011112E
:1040100072C075C09F3F19F09F5F9093E30118161F
:1040200024F40E94631E8093E5018091E50187FFDF
:1040300005C00E94631E81958093E5011C1624F43F
:104040000E94631E8093E6018091E60187FF05C010
:104050000E94631E81958093E6016091E5016623CD
:1040600039F1C091E601CC2319F1772767FD7095EE
:10407000872F972F0E94522323E333E343E35FE329
:104080000E94B6230E941F236093E5016C2F7727BF
:1040900067FD7095872F972F0E94522323E333E308
:1040A00043E35FE30E94B6230E941F236093E6016F
:1040B0001D1624F40E94AC1E8093E7018091E70155
:1040C00087FF05C00E94AC1E81958093E701111601
:1040D00024F40E94AC1E8093E8018091E80187FFE0
:1040E00005C00E94AC1E81958093E801DF91CF91BD
:1040F0001F910C94D21F9F3F09F08ECF96CFDF9176
:10410000CF911F910895E4EEF1E085E0DF011D926B
:104110008A95E9F71092E3011092E2010895833045
:1041200081F128F4813059F08230D1F00895853042
:1041300009F449C0B8F1863009F456C00895809159
:104140001501262F30E0280F311D2F3F310524F4B3
:10415000680F6093150108958FEF809315010895FE
:1041600080911401262F30E0280F311D2F3F31059B
:1041700024F4680F6093140108958FEF8093140165
:10418000089580911301262F30E0280F311D2F3F15
:10419000310524F4680F6093130108958FEF809325
:1041A0001301089580911201262F30E0280F311D50
:1041B0002F3F310524F4680F6093120108958FEFAB
:1041C00080931201089580911101262F30E0280F6D
:1041D000311D2F3F310524F4680F609311010895BC
:1041E0008FEF80931101089580911001262F30E008
:1041F000280F311D2F3F310524F4680F6093100103
:1042000008958FEF809310010895833011F128F401
:10421000813049F0823091F00895853081F120F1AC
:104220008630C1F1089580911501681720F4861B2E
:10423000809315010895109215010895809114013D
:10424000681720F4861B80931401089510921401BE
:10425000089580911301681720F4861B8093130141
:10426000089510921301089580911201681720F4A7
:10427000861B809312010895109212010895809177
:104280001101681720F4861B809311010895109284
:104290001101089580911001681720F4861B809306
:1042A000100108951092100108950F931F938D31FE
:1042B00009F46BC008F03FC08E3009F47FC0C0F431
:1042C000873009F469C068F4863009F0B1C0809184
:1042D000DA01817F8E7F8093DA0181E08093EA01A9
:1042E000A8C0883009F4A2C08B3009F49FC0A0C0D8
:1042F000863109F49BC078F4803109F472C08131B1
:1043000009F096C00E94251590910D0181E0892742
:1043100080930D018BC0893109F488C08B3109F07D
:1043200087C08091DA0181FB222720F991E0922752
:1043300090FB81F94CC0853309F470C048F4873292
:1043400009F46CC008F459C0893209F467C070C020
:10435000833438F48A3308F04EC0883309F466C0D9
:1043600067C0833409F45AC0883409F061C00E94E0
:1043700025150FEF13ED20E3015010402040E1F729
:1043800000C000000E94981C51C00E94D9220E94C7
:104390008C100E9485094AC09091DA01892F80957E
:1043A000817080FB90F929F0966098609093DA0113
:1043B00040C0997F977F9093DA0138C08091DA01ED
:1043C00082FB222720F991E0922790FB82F98093CB
:1043D000DA01992359F18091DA0181608093DA0141
:1043E00025C08091DA0183FB222720F991E09227F2
:1043F00090FB83F9ECCF895301C08D5141E050E02F
:1044000060E070E08A019B0104C0000F111F221FB1
:10441000331F8A95D2F7C901B80104C061E070E08A
:1044200080E090E00E94E5180E94251581E001C01F
:1044300080E01F910F91089580E0089580E0089535
:10444000CF93C82F8091EA01813079F018F0823043
:10445000E9F187C0E0910E01F0910F018081813177
:1044600069F0823209F07FC009C0E0910E01F0913D
:104470000F018081813111F0823261F48C2F0E9412
:104480001C22811104C08C2F0E9455211DC081E087
:1044900090E01AC08C2F0E941E22811114C0C431DA
:1044A00079F048F4CB3079F0C03109F060C082E097
:1044B0008093EA0108C0C93219F0C83321F057C00F
:1044C0001092EA0154C081E0817053C0C93289F171
:1044D00018F5C43171F1A8F4C73009F046C08AE07C
:1044E0008093150194E19093140193E0909313014C
:1044F0008093120188E08093110188E2809310017B
:1045000034C0CE51C63088F5EC2FF0E0E65DFE4FAA
:1045100080818093E90129C0CE34E9F020F4CB34C6
:1045200021F56AE013C0C13579F0C235F1F461E0DC
:104530000DC08091E901882319F01092E90115C09E
:1045400081E08093EA0115C061E006C08091E90135
:104550000E948F200AC06AE08091E9010E94052133
:1045600004C01092EA0180E004C081E002C080E053
:10457000ABCFCF910895E1E8F0E08081886080833F
:104580008081816080838FB7F89493E09093890055
:1045900090ED909388008FBF0895EFE6F0E0808162
:1045A000826080830895EFE6F0E080818D7F8083D4
:1045B0000895EFE6F0E0908182E0892780830895F6
:1045C0001F920F920FB60F9211242F933F934F9388
:1045D0005F936F937F938F939F93AF93BF93EF936B
:1045E000FF938091EB019091EC0101969093EC0187
:1045F0008093EB01811103C082E00E948509E09164
:10460000EC01E695E695F0E0E45AFA4FE4918091EA
:10461000EB018E1303C080E00E948509FF91EF91AA
:10462000BF91AF919F918F917F916F915F914F91CA
:104630003F912F910F900FBE0F901F90189504D0AF
:104640006894B1118DC0089570D088F09F5790F094
:10465000B92F9927B751A0F0D1F0660F771F881FA7
:10466000991F1AF0BA95C9F712C0B13081F077D00E
:10467000B1E0089574C0672F782F8827B85F39F0AC
:10468000B93FCCF3869577956795B395D9F73EF406
:1046900090958095709561957F4F8F4F9F4F0895AE
:1046A000E89409C097FB3EF49095809570956195CC
:1046B0007F4F8F4F9F4F9923A9F0F92F96E9BB2782
:1046C0009395F695879577956795B795F111F8CFFE
:1046D000FAF4BB0F11F460FF1BC06F5F7F4F8F4F69
:1046E0009F4F16C0882311F096E911C0772321F05F
:1046F0009EE8872F762F05C0662371F096E8862FF7
:1047000070E060E02AF09A95660F771F881FDAF74D
:10471000880F9695879597F9089557FD9058440FFF
:10472000551F59F05F3F71F04795880F97FB991F10
:1047300061F09F3F79F087950895121613061406CD
:10474000551FF2CF4695F1DF08C01616170618065A
:10475000991FF1CF86957105610508940895E89435
:10476000BB2766277727CB0197F908950BD078C030
:1047700069D028F06ED018F0952309F05AC05FC0B8
:104780001124EECFCADFA0F3959FD1F3950F50E02F
:10479000551F629FF001729FBB27F00DB11D639FF3
:1047A000AA27F00DB11DAA1F649F6627B00DA11D99
:1047B000661F829F2227B00DA11D621F739FB00D3F
:1047C000A11D621F839FA00D611D221F749F3327AF
:1047D000A00D611D231F849F600D211D822F762F48
:1047E0006A2F11249F5750408AF0E1F088234AF045
:1047F000EE0FFF1FBB1F661F771F881F9150504091
:10480000A9F79E3F510570F014C0AACF5F3FECF3AB
:10481000983EDCF3869577956795B795F795E7957C
:104820009F5FC1F7FE2B880F911D9695879597F98D
:10483000089597F99F6780E870E060E008959FEF22
:1048400080EC089500240A94161617061806090627
:10485000089500240A9412161306140605060895F6
:10486000092E0394000C11F4882352F0BB0F40F47E
:10487000BF2B11F460FF04C06F5F7F4F8F4F9F4FBE
:10488000089597FB072E16F4009407D077FD09D002
:104890000E945B2407FC05D03EF4909581959F4FC4
:1048A0000895709561957F4F0895EE0FFF1F059055
:1048B000F491E02D0994AA1BBB1B51E107C0AA1F6C
:1048C000BB1FA617B70710F0A61BB70B881F991FB1
:1048D0005A95A9F780959095BC01CD010895F99955
:1048E000FECF92BD81BDF89A992780B50895A8E1C1
:1048F000B0E042E050E00C949724262FF999FECFC7
:1049000092BD81BDF89A019700B4021639F01FBA22
:1049100020BD0FB6F894FA9AF99A0FBE0895019641
:10492000272F0E947E240C947D24DC01CB01FC0106
:10493000F999FECF06C0F2BDE1BDF89A319600B4F8
:0E4940000D9241505040B8F70895F894FFCF03
:10494E0002208709150AF209BE098A090101C70169
:10495E0028080A03140A3F4D36391D05D0049A045F
:10496E006104F4030D0426043F040102030405064A
:04497E00070809001D
:00000001FF
